S00F0000476174696C686F2E737265634D
S11300000EC01DC01CC01BC01AC019C018C017C028
S113001016C015C014C013C012C011C010C01124E2
S11300201FBECFE5D2E0DEBFCDBF20E0A0E6B0E04A
S113003001C01D92A536B207E1F715D27EC3E0CF09
S1130040CF92DF92EF92FF92CF93DF938091610082
S1130050813031F4B19B02C0C098FCCFC09AFACF72
S1130060823009F05EC089EF90E00197F1F700C09B
S11300700000C0E0B199F7CFCF5FE9EFF0E031972E
S1130080F1F700C00000C63008F449C0C09AB19925
S1130090F1CFC0E080916200C81788F4C1110DC08F
S11300A080E090916300891778F5E9EFF0E03197EB
S11300B0F1F700C000008F5FF4CFB19B02C0C0987D
S11300C025C0D0E06D2F70E080E090E005D26B0198
S11300D07C0180916300682F70E080E090E0FCD1A7
S11300E026E636E646E65FE356D29B01AC01C7013D
S11300F0B601ECD187FF08C089EF90E00197F1F7D2
S113010000C00000DF5FDECFCF5FC4CFE9EFF0E0D7
S11301103197F1F700C00000B19BF8CFABCFC09886
S1130120A9CF833009F077C089EF90E00197F1F708
S113013000C00000C0E0B199F7CFCF5FE9EFF0E075
S11301403197F1F700C00000C63008F462C0C09ACD
S1130150B199F1CFC0E080916200C817A8F5CC2313
S113016011F0D0E00DC080E090916300891750F544
S1130170E9EFF0E03197F1F700C000008F5FF4CFB2
S11301806D2F70E080E090E0A7D16B017C0180913D
S11301906300682F70E080E090E09ED126E636E6AA
S11301A046E65FE3F8D19B01AC01C701B6018ED1ED
S11301B087FF08C089EF90E00197F1F700C00000C5
S11301C0DF5FDECFCF5FC7CFB19923C0D0E06D2F03
S11301D070E080E090E080D16B017C01809163004D
S11301E0682F70E080E090E077D126E636E646E6B8
S11301F05FE3D1D19B01AC01C701B60167D187FF91
S1130200E3CFE9EFF0E03197F1F700C00000DF5FE2
S1130210DECFC09890CFDF91CF91FF90EF90DF9029
S1130220CF90089582E3C09A91E29A95F1F7000085
S1130230C098E9EFF0E03197F1F700C00000815079
S113024091F70895CF93DF9310926100EBDFB19B98
S1130250FDCFD1E010926400B19923C08091640075
S11302608F5F8093640087EA91E60197F1F700C0FD
S11302700000809164008F3178F3809161008430B4
S113028010F0D093610080916100811102C0D0937D
S113029061006091610070E08CE090E040D2C0E0C9
S11302A001C0C1E0809164008330F8F08F31C0F068
S11302B01092640090916400809161009817A8F4F2
S11302C0B1DF9FE9E6E8F1E09150E040F040E1F76A
S11302D000C00000809164008F5F80936400EACFC7
S11302E0809161008F5F80936100C111B3CF9ADF69
S11302F0B19BFDCF80916100813009F4B1C01092AF
S1130300640091E0B19920C0809164008F5F809374
S11303106400E9EFF0E03197F1F700C0000080914C
S11303206400863078F3C09A809164008F5F809374
S1130330640089EF90E00197F1F700C00000B19BE1
S1130340F3CFC09890E0DECF9111D9CF1092640022
S113035091E0B1992AC0809164008F5F809364001A
S1130360E9EFF0E03197F1F700C0000080916400FC
S1130370863078F3C09A809164008F5F8093640024
S113038089EF90E00197F1F700C00000B19BF3CF33
S1130390C0986091640070E08BE090E0C0D18091DF
S11303A064008093630090E0D4CF9111CFCF9FE39A
S11303B0EDE0F3E09150E040F040E1F700C00000D0
S11303C031DFB19BFDCF10926200D3E01092640044
S11303D0B1991DC0809164008F5F8093640087EAA7
S11303E091E60197F1F700C00000809164008F311D
S11303F078F380916200811102C0D0936200609111
S1130400620070E08AE090E08AD1C0E001C0C1E0FF
S1130410809164008330F8F08F31C0F01092640052
S113042090916400809162009817A8F4FBDE9FE924
S1130430E6E8F1E09150E040F040E1F700C0000050
S1130440809164008F5F80936400EACF80916200A2
S11304508F5F80936200C111B9CFE4DEB19BFDCF01
S1130460DF91CF910895B998B89AC098DBDE8FE4F4
S113047093EC0197F1F700C00000D4DE1092600005
S1130480809160008F5F8093600087EE93E0019716
S1130490F1F700C0000080916000B19902C0883C6F
S11304A078F3883C88F48AE090E031D1809362004C
S11304B08BE090E02CD1809363008CE090E027D116
S11304C080936100BDDDDACFBDDED8CF40D008F423
S11304D081E00895E89409C097FB3EF490958095D7
S11304E0709561957F4F8F4F9F4F9923A9F0F92FF6
S11304F096E9BB279395F695879577956795B79574
S1130500F111F8CFFAF4BB0F11F460FF1BC06F5F59
S11305107F4F8F4F9F4F16C0882311F096E911C06B
S1130520772321F09EE8872F762F05C0662371F08C
S113053096E8862F70E060E02AF09A95660F771FA0
S1130540881FDAF7880F9695879597F90895990F7C
S11305500008550FAA0BE0E8FEEF16161706E80789
S1130560F907C0F012161306E407F50798F0621BAA
S1130570730B840B950B39F40A2661F0232B242B7F
S1130580252B21F408950A2609F4A140A6958FEF9E
S1130590811D811D08950AD080C071D028F076D0C5
S11305A018F0952309F062C067C0ABC087D0A8F3E8
S11305B09923D9F35523C9F3950F50E0551FAA2762
S11305C0EE27FF27BB2700240894679520F4E20F49
S11305D0F31FB41F0A1E220F331F441FAA1F669560
S11305E0A9F7779530F4F30FB41F0A1E121E08F40E
S11305F06395330F441FAA1F221F769599F7879599
S113060020F4B40F0A1E121E631F440FAA1F221FD8
S1130610331F8695A9F7862F712D602D11249F57BE
S113062050408AF0E1F088234AF0EE0FFF1FBB1F11
S1130630661F771F881F91505040A9F79E3F5105B0
S113064070F014C05EC05F3FECF3983EDCF3869517
S113065077956795B795F795E7959F5FC1F7FE2B5B
S1130660880F911D9695879597F9089597F99F6737
S113067080E870E060E008959FEF80EC0895002426
S11306800A941616170618060906089500240A94F3
S113069012161306140605060895092E0394000C79
S11306A011F4882352F0BB0F40F4BF2B11F460FF08
S11306B004C06F5F7F4F8F4F9F4F089557FD905831
S11306C0440F551F59F05F3F71F04795880F97FB12
S11306D0991F61F09F3F79F08795089512161306CC
S11306E01406551FF2CF4695F1DF08C016161706FB
S11306F01806991FF1CF8695710561050894089530
S1130700E894BB2766277727CB0197F90895E199E9
S1130710FECF9FBB8EBBE09A99278DB30895262FF9
S1130720E199FECF1CBA9FBB8EBB2DBB0FB6F894CC
S1110730E29AE19A0FBE01960895F894FFCF65
S9030000FC
